:100000000C9461000C947E000C947E000C947E0095
:100010000C947E000C947E000C947E000C947E0068
:100020000C947E000C947E000C947E000C947E0058
:100030000C947E000C947E000C947E000C947E0048
:100040000C945A010C947E000C947E000C947E005B
:100050000C947E000C947E000C947E000C947E0028
:100060000C947E000C947E00000000002400270009
:100070002A0000000000250028002B0000000000DE
:1000800023002600290004040404040404040202DA
:100090000202020203030303030301020408102007
:1000A0004080010204081020010204081020000012
:1000B0000008000201000003040700000000000027
:1000C000000011241FBECFEFD8E0DEBFCDBF11E08E
:1000D000A0E0B1E0EAECFDE002C005900D92A43092
:1000E000B107D9F721E0A4E0B1E001C01D92AD3124
:1000F000B207E1F70E94A4010C94E3060C940000FF
:10010000833081F028F4813099F08230A9F008958D
:100110008730A9F08830C9F08430B1F48091800034
:100120008F7D03C0809180008F7780938000089539
:1001300084B58F7784BD089584B58F7DFBCF809182
:10014000B0008F778093B00008958091B0008F7DCC
:10015000F9CFCF93DF93282F30E0F901E255FF4F1D
:100160008491F901E656FF4FD491F901EA57FF4F08
:10017000C491CC23A1F081110E948000EC2FF0E00B
:10018000EE0FFF1FE458FF4FA591B491EC91ED23C2
:1001900081E090E009F480E0DF91CF91089580E064
:1001A00090E0FACF1F93CF93DF93282F30E0F9012F
:1001B000E255FF4F8491F901E656FF4FD491F901C2
:1001C000EA57FF4FC491CC23A9F0162F81110E944A
:1001D0008000EC2FF0E0EE0FFF1FEE58FF4FA591CF
:1001E000B4918FB7F894EC91111108C0D095DE232B
:1001F000DC938FBFDF91CF911F910895DE2BF8CF55
:10020000CF93DF9390E0FC01E656FF4F24918A578D
:100210009F4FFC0184918823C9F090E0880F991FBB
:10022000FC01E859FF4FA591B491FC01EE58FF4F36
:10023000C591D49161110DC09FB7F8948C91209510
:1002400082238C938881282328839FBFDF91CF91BD
:100250000895623051F49FB7F8943C91822F8095B5
:1002600083238C93E8812E2BEFCF8FB7F894EC91FA
:100270002E2B2C938FBFEACF8E50806480937C000E
:1002800080917A00806480937A0080917A0086FD64
:10029000FCCF809178009091790008952FB7F89461
:1002A0006091190170911A0180911B0190911C01BC
:1002B0002FBF08951F920F920FB60F9211242F9304
:1002C0003F938F939F93AF93BF9380911901909128
:1002D0001A01A0911B01B0911C013091180123E07B
:1002E000230F2D3758F50196A11DB11D209318013C
:1002F0008093190190931A01A0931B01B0931C01E4
:100300008091140190911501A0911601B0911701EF
:100310000196A11DB11D8093140190931501A09326
:100320001601B0931701BF91AF919F918F913F91AB
:100330002F910F900FBE0F901F90189526E8230F56
:100340000296A11DB11DD2CFCF93DF9300D000D074
:10035000CDB7DEB7789484B5826084BD84B5816002
:1003600084BD85B5826085BD85B5816085BD809180
:100370006E00816080936E001092810080918100F8
:1003800082608093810080918100816080938100F0
:10039000809180008160809380008091B1008460B2
:1003A0008093B1008091B00081608093B000809113
:1003B0007A00846080937A0080917A0082608093D2
:1003C0007A0080917A00816080937A0080917A002F
:1003D000806880937A001092C10060E081E10E9401
:1003E000000162E084E00E94000161E08BE00E9475
:1003F000000161E083E00E94000160E089E00E946A
:10040000000160E08EE00E94000160E08BE00E944D
:10041000D20024E6422E512C612C712C80E10E94E6
:100420003C019C838B8381E02B813C8121153240F0
:100430000CF480E080931301809112018823A9F0CD
:100440002B813C81211532400CF4B4C10E944E0135
:10045000683E73408105910540F060E083E00E94B2
:10046000D20010921201109211018EE00E943C0104
:100470008C0183E10E943C010B5F1F4F080F191F85
:100480000F3F13400CF066C08EE00E943C018C01CF
:1004900083E10E943C010B5F1F4F080F191F8FE083
:1004A0000E943C018A3F93400CF057C08FE00E94AD
:1004B0003C010596BC01990F880B990B0E94990588
:1004C00020E030EC4FE754E40E94EF046B017C0124
:1004D000B801110F880B990B0E94990520E030ECB0
:1004E0004FE754E40E94EF044B015C012B813C81F7
:1004F000B901330F880B990B0E94990520E030EC6D
:100500004FE754E40E94EF0420E030E040E05FE376
:100510000E94490608E010E0181614F400E110E00B
:1005200020E030E0A901C501B4010E94EA0487FF80
:1005300017C0B801012E000C880B990B0E94990579
:1005400020E030E0A9010E944E060E9461057C83F4
:100550006B832AC00FEF13E0A2CF8FEF93E0AACFF7
:1005600020E030E040E85FE3C501B4010E944906A5
:10057000181634F4812C912C90E8A92E9FE3B92E03
:10058000B801012E000C880B990B0E949905A5015A
:1005900094010E944E060E9461057C836B830617BE
:1005A000170714F41C830B8320E030E0A901C70176
:1005B000B6010E94EA0487FDF2C020E030E040E886
:1005C0005FE3C701B6010E94490618160CF4EBC0A0
:1005D00089E00E94A90021E02A838130910509F079
:1005E0001A82019709F06DC080911001811169C0D4
:1005F000309111013983311164C00E942F044B01E5
:100600005C0180910E0190910F018017910724F0F9
:1006100010920F0110920E0120900E0130900F01E8
:100620008B819C81181619065CF58017910794F44C
:100630009C01229DC001239D900D329D900D11249F
:10064000B8010E94BB06009729F0820F931F08177C
:100650001907B4F4C501B401A30192010E948704F3
:100660000E94990520E030E048EC52E40E94EF043B
:10067000A70196010E94EA04881F8827881F8983A2
:10068000C1010196B8010E94BB0690930F018093AF
:100690000E0139813323A9F061E08BE00E94D20082
:1006A00061E083E00E94D2000E944E0160930A0143
:1006B00070930B0180930C0190930D0181E0809366
:1006C000090181E10E94A9008C0184E00E94A90037
:1006D0009C838B830130110511F0892B69F5809182
:1006E0000801811121C00E944E01C0900401D090E8
:1006F0000501E0900601F09007016C197D098E0953
:100700009F09633371058105910570F00E944E01C8
:100710006093040170930501809306019093070193
:1007200010920F0110920E0181E00130110529F0A5
:100730002B813C81232B09F080E0809308013A81D2
:100740003093100180910901882309F10E944E0124
:1007500000910A0110910B0120910C0130910D01C3
:10076000601B710B820B930B6A307105810591053B
:1007700070F060E08BE00E94D20080911101811145
:1007800004C060E083E00E94D2001092090180E082
:1007900090E0892B09F442CE0E9400003FCEC12C8C
:1007A000D12C760115CFC12CD12C80E8E82E8FE317
:1007B000F82E0ECF0E944E01643F714081059105D5
:1007C00008F453CE4ACE8F929F92AF92BF92CF92AF
:1007D000DF92EF92FF92CF93DF93EC0168817981F2
:1007E0008A819B81611571058105910521F464E27F
:1007F00079ED8BE597E02DE133EF41E050E00E9489
:10080000870449015A019B01AC01A7EAB1E40E94A7
:10081000A6046B017C01ACEEB4EFA50194010E942B
:10082000B404C60ED71EE81EF91EF7FE06C081E00E
:10083000C81AD108E10880E8F80AC882D982EA8299
:10084000FB82C701B6019F77DF91CF91FF90EF90B8
:10085000DF90CF90BF90AF909F908F9008958F9230
:100860009F92AF92BF92CF92DF92EF92FF926091F0
:1008700000017091010180910201909103016115C5
:1008800071058105910521F464E279ED8BE597E02E
:100890002DE133EF41E050E00E94870449015A0105
:1008A0009B01AC01A7EAB1E40E94A6046B017C01A4
:1008B000ACEEB4EFA50194010E94B404C60ED71E9D
:1008C000E81EF91EF7FE06C081E0C81AD108E1084B
:1008D00080E8F80AC0920001D0920101E092020182
:1008E000F0920301C701B6019F77FF90EF90DF9070
:1008F000CF90BF90AF909F908F900895609300012C
:100900007093010180930201909303010895052ED5
:1009100097FB1EF400940E949E0457FD07D00E948E
:10092000B90407FC03D04EF40C949E0450954095F6
:10093000309521953F4F4F4F5F4F0895909580958B
:10094000709561957F4F8F4F9F4F08950E94DB04F4
:10095000A59F900DB49F900DA49F800D911D112413
:100960000895B7FF0C94A6040E94A604821B930B63
:100970000895A1E21A2EAA1BBB1BFD010DC0AA1FE0
:10098000BB1FEE1FFF1FA217B307E407F50720F0F8
:10099000A21BB30BE40BF50B661F771F881F991F73
:1009A0001A9469F760957095809590959B01AC01BC
:1009B000BD01CF010895A29FB001B39FC001A39FC5
:1009C000700D811D1124911DB29F700D811D112488
:1009D000911D08950E94D40508F481E008950E94B5
:1009E00003050C940F060E94080658F00E940106A9
:1009F00040F029F45F3F29F00C94F80551110C9454
:100A000043060C94FE050E94200668F39923B1F377
:100A1000552391F3951B550BBB27AA276217730724
:100A2000840738F09F5F5F4F220F331F441FAA1FB8
:100A3000A9F335D00E2E3AF0E0E832D09150504074
:100A4000E695001CCAF72BD0FE2F29D0660F771F22
:100A5000881FBB1F261737074807AB07B0E809F008
:100A6000BB0B802DBF01FF2793585F4F3AF09E3F8D
:100A7000510578F00C94F8050C9443065F3FE4F3BD
:100A8000983ED4F3869577956795B795F7959F5FD0
:100A9000C9F7880F911D9695879597F90895E1E01C
:100AA000660F771F881FBB1F621773078407BA077B
:100AB00020F0621B730B840BBA0BEE1F88F7E095D6
:100AC00008950E9468056894B1110C944306089536
:100AD0000E94280688F09F5798F0B92F9927B751A0
:100AE000B0F0E1F0660F771F881F991F1AF0BA95D2
:100AF000C9F714C0B13091F00E944206B1E00895E8
:100B00000C944206672F782F8827B85F39F0B93FD9
:100B1000CCF3869577956795B395D9F73EF4909584
:100B20008095709561957F4F8F4F9F4F0895E89402
:100B300009C097FB3EF490958095709561957F4F25
:100B40008F4F9F4F9923A9F0F92F96E9BB279395D3
:100B5000F695879577956795B795F111F8CFFAF4E3
:100B6000BB0F11F460FF1BC06F5F7F4F8F4F9F4F14
:100B700016C0882311F096E911C0772321F09EE872
:100B8000872F762F05C0662371F096E8862F70E0D8
:100B900060E02AF09A95660F771F881FDAF7880FB2
:100BA0009695879597F90895990F0008550FAA0B08
:100BB000E0E8FEEF16161706E807F907C0F0121670
:100BC0001306E407F50798F0621B730B840B950B73
:100BD00039F40A2661F0232B242B252B21F40895C8
:100BE0000A2609F4A140A6958FEF811D811D089565
:100BF00097F99F6780E870E060E008959FEF80ECD0
:100C0000089500240A941616170618060906089572
:100C100000240A9412161306140605060895092ED8
:100C20000394000C11F4882352F0BB0F40F4BF2B47
:100C300011F460FF04C06F5F7F4F8F4F9F4F089587
:100C400057FD9058440F551F59F05F3F71F047957D
:100C5000880F97FB991F61F09F3F79F08795089562
:100C6000121613061406551FF2CF4695F1DF08C081
:100C7000161617061806991FF1CF8695710561059E
:100C800008940895E894BB2766277727CB0197F946
:100C900008950E94D40508F48FEF08950E9461061C
:100CA0000C940F060E94010638F00E94080620F0FE
:100CB000952311F00C94F8050C94FE0511240C9466
:100CC00043060E94200670F3959FC1F3950F50E0F4
:100CD000551F629FF001729FBB27F00DB11D639FEE
:100CE000AA27F00DB11DAA1F649F6627B00DA11D94
:100CF000661F829F2227B00DA11D621F739FB00D3A
:100D0000A11D621F839FA00D611D221F749F3327A9
:100D1000A00D611D231F849F600D211D822F762F42
:100D20006A2F11249F5750409AF0F1F088234AF01F
:100D3000EE0FFF1FBB1F661F771F881F915050408B
:100D4000A9F79E3F510580F00C94F8050C944306DA
:100D50005F3FE4F3983ED4F3869577956795B79512
:100D6000F795E7959F5FC1F7FE2B880F911D96952C
:100D7000879597F9089597FB072E16F4009407D0EE
:100D800077FD09D00E94CF0607FC05D03EF4909570
:100D900081959F4F0895709561957F4F0895AA1B87
:100DA000BB1B51E107C0AA1FBB1FA617B70710F056
:100DB000A61BB70B881F991F5A95A9F78095909588
:0A0DC000BC01CD010895F894FFCFA7
:040DCA000100000024
:00000001FF
